:100000000C944C000C9469000C9469000C946900E9
:100010000C9469000C9469000C9469000C946900BC
:100020000C9469000C94BB000C9469000C9469005A
:100030000C9469000C9469000C9469000C9469009C
:100040000C9469000C942C030C94F7010C94B301EC
:100050000C949E010C9469000C9469000C94690046
:100060000C9469000C946900205B253032785D0A9D
:10007000006374726C5F616C6C6F63282564292067
:100080006964783D25640A007E0E0E0E0E1B1B1C53
:100090000E1B1B7E0E0E0E0E11241FBECFEFD4E0E2
:1000A000DEBFCDBF11E0A0E0B1E0EAECF8E202C0B3
:1000B00005900D92A231B107D9F713E0A2E1B1E0AA
:1000C00001C01D92A433B107E1F70E9474000C94A3
:1000D00063140C940000809112010895A8950E9469
:1000E00080030E9432100895F894A8950E9454014C
:1000F0000E94F2020E94FE0E8FEF80931001409A40
:100100000E947A01789480E090E060E040E050E066
:100110000E94861080E090E00E94350F0E94DB0C68
:100120000E9498020E942E080E946E00F9CF9091C2
:1001300012019817F1F09630E1F0953011F4863005
:10014000C1F4809312010E946804809112018530ED
:1001500029F480E060E245E00E942D1180911201B7
:10016000863029F480E060E246E00E942D1181E0B3
:10017000089580E008951F920F920FB60F921124F8
:100180008F939F93AF93BF9380912A03882329F085
:1001900080912A03815080932A0380911301882340
:1001A00029F581E0809313017894809114018F5F89
:1001B000809314018091140190E083709070892BDA
:1001C00099F48091260390912703A0912803B09180
:1001D00029030196A11DB11D809326039093270347
:1001E000A0932803B093290310921301BF91AF91FC
:1001F0009F918F910F900FBE0F901F9018951092A6
:100200002603109227031092280310922903E0E797
:10021000F0E010821092B00082E08093B100808103
:10022000816080830895EF92FF920F931F93209136
:1002300026033091270340912803509129037C0124
:1002400000E010E0E20EF31E041F151F02C00E9422
:100250006E00C801B7010E9448118823C1F31F91A5
:100260000F91FF90EF900895EF92FF920F931F93DD
:1002700020912603309127034091280350912903B0
:100280007C0100E010E0E20EF31E041F151F01C008
:10029000A895C801B7010E9448118823C9F31F918E
:1002A0000F91FF90EF900895EAEFFFE39491892F6B
:1002B00081508E3F10F4909366000895ECEFFFE3B9
:1002C00025913591459154915070B901CA01089515
:1002D000EFEFFFE3E4918E2F0895F8942CE088E18E
:1002E00090E00FB6F894A895809360000FBE20931D
:1002F0006000FFCF1092160180911601E6E1F1E057
:1003000082938081809330018091300180932F010E
:10031000519A5098599A589A5A9882E08093C000FE
:100320001092C5008FE08093C40086E08093C200E5
:100330008CEF8093C10080E090E008951F920F92AF
:100340000FB60F9211248F9310921601809116010F
:10035000809315015A988091C6008F910F900FBE1F
:100360000F901F9018951F920F920FB60F921124A5
:100370008F939F93EF93FF9390912F018091300182
:10038000981731F48091C1008F7D8093C10026C001
:100390005A9A8091390187FF09C0809139018F777E
:1003A000809339018091C100816003C08091C100B8
:1003B0008E7F8093C100E0913001F0E0EB5EFE4F54
:1003C000848D8093C600809130018F5F80933001CF
:1003D00080913001883010F010923001FF91EF9140
:1003E0009F918F910F900FBE0F901F9018951F92A5
:1003F0000F920FB60F9211242F933F938F939F93D9
:10040000EF93FF935A9B03C08091C60030C02091A8
:1004100015018091160130E090E001972817390707
:1004200041F080911501873179F48091160188237C
:1004300059F4809116018F5F809316018091160107
:10044000883110F010921601E0911501F0E08091D2
:10045000C600EB5EFE4F8283809115018F5F809313
:10046000150180911501883110F010921501FF914E
:10047000EF919F918F913F912F910F900FBE0F9011
:100480001F901895482FA89507C08091C1008062E1
:100490008093C1007894A89520912F01809130011C
:1004A00030E090E001972817390779F380912F0108
:1004B000873021F480913001882339F3E0912F01B6
:1004C000F0E0EB5EFE4F448F80912F018F5F8093B1
:1004D0002F0180912F01883010F010922F01809110
:1004E000C10080628093C100842F0895282F5A99FB
:1004F000FECF8091390180688093390110921601F6
:1005000080911601809315012F77A22FA295AF70CD
:10051000B0E0A050BF4FE22FF0E0EF70F070E0507D
:10052000FF4F8C9190818927822B0E94420208956F
:100530005A991CC090911501809116019817B1F03D
:10054000E0911601F0E0EB5EFE4F9281F89480910D
:1005500016018F5F8093160180911601883110F08B
:1005600010921601292F30E0789402C02FEF3FEF50
:10057000C90108958BB190E09695879596958795DA
:1005800081700895EF92FF920F931F939C011816AC
:1005900019061CF58091260390912703A09128034A
:1005A000B091290379010027F7FC0095102FE80E80
:1005B000F91E0A1F1B1F8091C100877F8093C10015
:1005C0005A9A599A02C00E946E00C801B7010E944F
:1005D00048118823C1F30E947A011F910F91FF9067
:1005E000EF9008951092C1001DBA10926800EDE6D8
:1005F000F0E010828081ECE6F0E0808380818093DF
:100600006B0093E09CBB87E08BBB1CBC94B915B816
:1006100081E087B98EE388B98EEF8AB99BB90E94D1
:10062000FF00A8952EE088E190E00FB6F894A89519
:10063000809360000FBE20936000089584B1837C96
:1006400084B985B1837C85B984EE8CBD01C08EB53B
:100650000DB407FCFCCF08951F920F920FB60F92B6
:1006600011242F933F934F935F936F937F938F93B7
:100670009F93AF93BF93EF93FF9380912B03909140
:100680002C032FEF8F3F920779F0249A8EBD0DB483
:1006900006FE03C024980E946E0E8FEF9FEF90938A
:1006A0002C0380932B0301C024988EB50E94630D08
:1006B0008DB59EB587FDFCCF86FDFACFFF91EF91FA
:1006C000BF91AF919F918F917F916F915F914F916A
:1006D0003F912F910F900FBE0F901F901895809112
:1006E000260390912703A0912803B09129038093BA
:1006F0003A0190933B01A0933C01B0933D010895D2
:10070000809110018F3F09F160913A0170913B0196
:1007100080913C0190913D01611571058105910524
:10072000B1F06C507E4F8F4F9F4F0E94481188232D
:1007300071F0409A8FEF8093100110923A0110925D
:100740003B0110923C0110923D0180E0089581E050
:10075000089580E090E060E040E050E00E94861064
:1007600040988091260390912703A0912803B0918F
:10077000290380933A0190933B01A0933C01B093ED
:100780003D0108950F931F93CF93DF938C010E9437
:10079000BE0CFC01D80112962C91129713968C91E5
:1007A0001397C82FD0E0D695DC2FCC27D795C795C7
:1007B000822F90E0C82BD92B11968C91853081F037
:1007C000863018F48330E9F405C0893079F080323E
:1007D000C1F415C0822F0E94970013C00E946707C2
:1007E000CE010E94C30C0097C9F70BC0309749F0A7
:1007F000D283C183D80114968C91838302C00E9456
:100800006D0180912D03882381F0F801208130E073
:100810002F7730708091100190E02817390729F464
:1008200080912D03815080932D03DF91CF911F91F3
:100830000F910895FC018181893159F02091C20105
:100840003091C3012115310551F0CF01F90109950E
:10085000089584818093C90181E08093C80108953F
:10086000CF93DF93E9012091C00192E1299FF0012C
:100870001124EC5AFE4F682B608342834F70DF01D6
:10088000139603C089918D9341504423D9F783E097
:1008900081838091C0018F5F8093C0018091C001EE
:1008A000863010F01092C0019091C0018091C1017A
:1008B000981759F48091C1018F5F8093C101809195
:1008C000C101863010F01092C101DF91CF910895DF
:1008D000DF93CF93CDB7DEB72F970FB6F894DEBF77
:1008E0000FBECDBF0E946B00833061F0843061F099
:1008F0009E012F5F3F4F823081F4198280E660E0D5
:1009000041E80FC081E001C082E0898380E660E0B9
:1009100041E69E012F5F3F4F04C0198280E660E0F0
:1009200041E60E9430042F960FB6F894DEBF0FBE4A
:10093000CDBFCF91DF910895DF92EF92FF920F9399
:100940001F93CF93DF93EC01062F7A012115310518
:1009500019F42FEF3FEF43C0C9010E94350F909368
:10096000C3018093C201D093C501C093C40110920A
:10097000C8018EEF9FEF9093C7018093C60110E0EE
:1009800084E0D82E002329F080E0602FA7010E9488
:100990001711D0922D0302C00E946E008091C801F1
:1009A000882321F480912D038823B1F70E942D0F15
:1009B000811110E08091C801882319F41F5F18305D
:1009C00008F38091C2019091C3010E94350F1092EB
:1009D000C3011092C2012091C6013091C701C90123
:1009E000DF91CF911F910F91FF90EF90DF900895CD
:1009F000EF92FF920F931F93DF93CF9300D000D01D
:100A000000D0CDB7DEB78C017E010894E11CF11C4B
:100A100086E0F70111928A95E9F7F8018385807FD6
:100A20008387C7010E940B11C8016EE0A7012BE963
:100A300035E00E949C0426960FB6F894DEBF0FBEE8
:100A4000CDBFCF91DF911F910F91FF90EF9008954F
:100A5000EF92FF920F931F93DF93CF9300D000D0BC
:100A600000D0CDB7DEB78C01FC01618172817E01BF
:100A70000894E11CF11CC7010E940B11F80164816C
:100A80006095607845815681C7010E94F41080E02E
:100A900063E0A7010E941711F80164816078458125
:100AA0005681C7010E94F41080E063E0A7010E9414
:100AB000171126960FB6F894DEBF0FBECDBFCF91AB
:100AC000DF911F910F91FF90EF900895EF92FF92A9
:100AD0000F931F93DF93CF9300D000D000D0CDB7FA
:100AE000DEB78C01FC01618172817E010894E11CFA
:100AF000F11CC7010E940B11F80145815681C70105
:100B000064810E94F41080E063E0A7010E94171145
:100B100088E0F801818783858F77838726960FB6D3
:100B2000F894DEBF0FBECDBFCF91DF911F910F9123
:100B3000FF90EF900895EF92FF920F931F93CF9342
:100B4000DF93FC01C091C401D091C501209721F42D
:100B500081E08093C801BCC08381282F30E03695A6
:100B6000322F222737952795828190E0282B392B29
:100B70008181893081F08A3020F4873008F4A8C060
:100B800011C08D3009F465C08D3008F4A1C08031EA
:100B900008F09EC007C03A83298384818B838B85AC
:100BA000846094C09581668177818F3011F08830A0
:100BB00019F48B8582608AC03A832983392F330FD9
:100BC000330F20E0442737FD4095542F8D819E81BF
:100BD000AF81B88580709070282B392B4A2B5B2B06
:100BE000862F90E08F779070A3E0880F991FAA95C9
:100BF000E1F7AA2797FDA095BA2F282B392B4A2B6E
:100C00005B2B872F90E08077907064E095958795B7
:100C10006A95E1F7AA2797FDA095BA2F282B392BC3
:100C20004A2B5B2B2D833E834F835887858190E031
:100C300080749070880F991F2481282B2C832B851A
:100C4000822F81608B87878180FD51C023602B8735
:100C50004EC0848190E0A0E0B0E08F779070A070EB
:100C6000B0708C01FF24EE24268130E040E050E09B
:100C70007EE1220F331F441F551F7A95D1F78D81D6
:100C80009E81AF81B885A070B070282B392B4A2B7C
:100C90005B2B2E293F29402B512B858190E0A0E032
:100CA000B0E08F779070A070B07067E1880F991FE7
:100CB000AA1FBB1F6A95D1F7282B392B4A2B5B2B18
:100CC0002D833E834F8358878B8588608B870FC029
:100CD0002091C2013091C3012115310521F0CF01CE
:100CE000F90109950FC0CF010E94C2030BC08B858B
:100CF0008F708F3039F481E08093C8011092C70162
:100D00001092C601DF91CF911F910F91FF90EF904C
:100D10000895EF92FF920F931F93CF93DF93162FB7
:100D2000E42E052F0E947602812F0E944202F82EA7
:100D30001F702E2D302FC901EC0104C089910E9433
:100D40004202F8269E012E192117C0F38F2D0E9412
:100D5000420200D000D0EDB7FEB7319688E690E0B1
:100D6000ADB7BEB712969C938E931197F282138201
:100D70000E9489110F900F900F900F90DF91CF91EB
:100D80001F910F91FF90EF900895DF93CF93CDB710
:100D9000DEB72F970FB6F894DEBF0FBECDBF6D89BB
:100DA000762F7F70CE014696DC0120E030E0AE0168
:100DB0004F5F5F4F08C0FA01E20FF31F8C918083F1
:100DC0002F5F3F4F12967217B1F78C890E948906E8
:100DD0002F960FB6F894DEBF0FBECDBFCF91DF9137
:100DE00008951F93CF93DF93182FEB018B810E94FF
:100DF0007F11982F8B3120F08D3120F08E3721F02C
:100E0000A0E003C0A2E001C0A4E08985883009F019
:100E1000A860EC816E2F6F779B51923078F461114E
:100E20006D5F862F90E08170907074E0880F991F3D
:100E30007A95E1F766956F70682B02C061116F5F5C
:100E40002D813E814F815885C90181709070892B19
:100E500011F470E001C070E1E0786E2B8DB79EB7A1
:100E60000A970FB6F8949EBF0FBE8DBFEDB7FEB7C1
:100E700031961066CDB7DEB7198384EE8183A283E5
:100E8000138264831582DA01C9018E719070A0709B
:100E9000B070B695A79597958795782B768317822E
:100EA00015E056954795379527951A95D1F72087E0
:100EB00011860E94C5068DB79EB70A960FB6F894A4
:100EC0009EBF0FBE8DBFDF91CF911F9108950F93ED
:100ED0001F93DF93CF93CDB7DEB72F970FB6F8945C
:100EE000DEBF0FBECDBF8C010097F1F080E4898397
:100EF000F80121813281832F992787FD9A95982FB8
:100F00008A832436310514F0906C9A83F80181812C
:100F10008B838081806663EEAE014F5F5F4F0E94DE
:100F2000890687E0F80182872F960FB6F894DEBF16
:100F30000FBECDBFCF91DF911F910F910895BF924A
:100F4000CF92DF92EF92FF920F931F93DF93CF9395
:100F500000D000D000D0CDB7DEB77C016B01009788
:100F600009F46BC06115710509F467C0DC011196C5
:100F70008D919C91129719962C918617970719F4C9
:100F8000283059F458C0283019F487E0F7018187D8
:100F9000D7011296DC92CE921197C6010E94C30C23
:100FA000FC01009719F18E159F0501F18181928155
:100FB000D70112969C938E931197838113968C93ED
:100FC0001397848114968C931497258136814781D9
:100FD000508515962D933D934D935C931897CF01B3
:100FE0000E94670788E0F701828725C0F6E0BF2EE0
:100FF0008E010F5F1F4FD801EB2D1D92EA95E9F787
:10100000D7011B968C911B97807F1B968C93C801F0
:10101000B6010E940B11C70161E0A8012BE935E080
:101020000E949C0497FF03C0F701B28606C088E0C7
:10103000D7011A968C9381E001C080E026960FB606
:10104000F894DEBF0FBECDBFCF91DF911F910F91FE
:10105000FF90EF90DF90CF90BF900895DF92EF92D6
:10106000FF920F931F93DF93CF9300D000D000D057
:10107000CDB7DEB7AC012FEF8F3F920769F184E166
:1010800080932A0380913E01882329F41092530112
:10109000109252014EC420915201213168F4E22F86
:1010A000F0E0EF5BFE4F40838091530184278093F3
:1010B00053012F5F2093520120915201223008F4F6
:1010C00038C430E08091410190E08F7090700296BA
:1010D0002817390709F02DC40E94BA02882319F095
:1010E00084E180932A0380912A038823E1F011E0B0
:1010F00015C0812F60E00E94E30CFC01009751F0C5
:101100008185883039F4838587FF04C0CF010E9430
:1011100066050FC41F5F1F3109F40BC40E947F0EC8
:1011200004973CF706C440915201242F30E080918F
:10113000410190E08F70907002962817390709F0EE
:1011400051C380915301882309F04CC30E943F0F83
:10115000D0903E018F3F81F400D000D0EDB7FEB7B4
:10116000319630E6D32AADB7BEB71196DC9281E650
:10117000818381E890E048C3409A8D2D61E00E9410
:10118000290D8C01009709F4FCC2FC018185863091
:1011900081F400D000D0EDB7FEB7319620E6D22A18
:1011A000ADB7BEB71196DC9281E6818381E890E00D
:1011B000F7C2823018F482E0F801818790914101F2
:1011C000892F82958F70853009F4F2C0863030F413
:1011D000823071F0843009F0D4C275C0893009F4CE
:1011E00049C28E3009F413C1883009F0CAC209C15E
:1011F000903221F4D8011A961C92DAC280914201F1
:10120000843259F1853220F4813209F0B2C207C02C
:10121000803809F445C0813809F0ABC249C0EDB748
:10122000FEB738970FB6F894FEBF0FBEEDBF3196EC
:1012300020E6D22AADB7BEB71196DC9283E6818351
:1012400081E290E09383828386E390E095838483B8
:1012500081E090E097838683C4C10E946B00823056
:1012600011F421E009C0882311F422E005C0843084
:1012700011F428E001C020E000D000D000D0EDB78C
:10128000FEB7319630E6D32AADB7BEB71196DC92E1
:1012900082E6818382E290E093838283248381C00B
:1012A0000E946B00882341F080E060E240E0ACC027
:1012B0000E946B00833019F40E94680479C280E0B8
:1012C00060E243E0A1C080914201E82EFF24EE0CD1
:1012D000FF1CEE0CFF1C8091430180FF04C0E2E084
:1012E000F0E0EE0EFF1EE1FC02C010E001C010E1D4
:1012F00081E491E0B7010E940B1180E090E069E188
:1013000041E451E02AE134E00E949C048091C9014B
:10131000823551F083351CF4873459F408C0873680
:1013200039F0823731F401C01068116002C01068D2
:101330001260B7016F5F7F4F81E491E00E940B1153
:1013400080E090E069E141E451E02AE134E00E946C
:101350009C048091C901823551F083351CF4873497
:1013600059F408C0873639F0823731F401C010686B
:10137000146002C01068186000D000D000D0EDB733
:10138000FEB7319620E6D22AADB7BEB71196DC92F1
:1013900082E48183F694E794F694E794F382E28200
:1013A000148315820E94C506EDB7FEB736961EC19E
:1013B0006091420170E093E0660F771F9A95E1F724
:1013C0000091430110E0C80187709070682B792B61
:1013D00081E090E0682779277E010894E11CF11CE8
:1013E000C7010E940B111B8283E0169507958A9511
:1013F000E1F701700C8380E066E0A7010E941711FD
:10140000D7C180E060E242E00E942D11D1C19091ED
:10141000430180E020914401E22EFF24E82AF92ACA
:101420002FEF3FE3E222F322809142018331A8F4BF
:10143000813108F0E1C0883009F482C0893030F48D
:101440008823D9F0873009F094C160C0893009F44D
:101450009DC0803109F08DC1F7C0803209F415C1FB
:10146000813220F4833109F084C1F3C0813209F460
:101470003FC1823209F07DC158C1D80111968D91CA
:101480009C911297E816F906A1F119968C9119977B
:10149000883019F487E019968C93C7010E94C30C19
:1014A000FC010097E9F080179107D1F081819281CA
:1014B000D80112969C938E931197838113968C93E7
:1014C0001397848114968C9385819681A781B0852A
:1014D000F80185839683A783B08787E0818704C05E
:1014E000C801B7010E94F8048D2DB8010E94F106D1
:1014F0005FC18D2DB8010E94F106D80111966D9142
:101500007C911297C8010E94F80452C1EDB7FEB752
:1015100038970FB6F894FEBF0FBEEDBF319620E6A8
:10152000D22AADB7BEB71196DC9283EE818380E5F7
:1015300090E093838283158214821782168251C0B1
:101540002DB73EB72A5030400FB6F8943EBF0FBEBD
:101550002DBFEDB7FEB7319630E6D32AADB7BEB793
:101560001196DC9284EE818381E590E093838283FF
:1015700015821482178216828FE090E0918780870F
:101580000E94C506EDB7FEB73A9630C0D801159651
:101590004D915D916D917C911897EDB7FEB738979D
:1015A0000FB6F894FEBF0FBEEDBF319620E6D22AEB
:1015B000ADB7BEB71196DC9223EE218322E530E071
:1015C00033832283BDE07695679557954795BA9505
:1015D000D1F744831582BB27A72F962F852F8683AB
:1015E00017820E94C506EDB7FEB738960FB6F8947D
:1015F000FEBF0FBEEDBFDCC0C801B7010E949F0750
:10160000882309F4D5C040914501842F90E09C01C6
:101610002071307054E0359527955A95E1F78F7019
:101620009070880F991F282B822F8150823028F4C8
:101630004078D80114964C931DC021112350407856
:10164000242BF801248391C0809145018F788093E9
:101650004501C801B7010E949F07882309F4A8C06B
:1016600090914501892F8F77813041F49078D8018E
:1016700014969C93C8010E9428059AC0811181503C
:101680009078892BF801848370C0C801B7010E944B
:101690009F07882309F48CC080914501D8011596D5
:1016A0002D913D914D915C91189784FF07C0216069
:1016B000F801258336834783508708C02E7FD801E1
:1016C00015962D933D934D935C931897809145010A
:1016D00090E08F709070880F991FAA2797FDA095B2
:1016E000BA2FF8012581368147815085217E35C08A
:1016F000C801B7010E949F07882309F459C080914F
:10170000450190E08F709070B5E0880F991FBA95F1
:10171000E1F7AA2797FDA095BA2FF8012581368118
:10172000478150852F713E7F18C0C801B7010E94C4
:101730009F078823E9F18091450190E08F709070B8
:10174000982F8827990FAA2797FDA095BA2FF801FF
:101750002581368147815085317E822B932BA42BA6
:10176000B52B85839683A783B087C8010E94660541
:101770001FC000D000D0EDB7FEB7319620E6D22AC8
:1017800007C000D000D0EDB7FEB73196B0E6DB2A37
:10179000ADB7BEB71196DC9281E6818382E890E016
:1017A000938382830E94C5060F900F900F900F9035
:1017B000409880913E0160E00E94E30C8C0100970C
:1017C00059F1FC018385806883870E947F0E03970F
:1017D0001CF1D80119968C918830F1F4C8010E944F
:1017E00066051AC04423C1F000D000D0EDB7FEB7A3
:1017F000319680913E018066ADB7BEB711968C934D
:1018000081E6818380E890E0938382830E94C5060D
:101810000F900F900F900F90109253011092520161
:1018200011E00CE0812F60E00E94E30CFC010097C6
:1018300069F08285882351F0893031F4DF01202F4F
:101840001D922A95E9F702C0818712861F5F103228
:1018500049F70E94BA02882309F06BC09091C00139
:101860008091C101981729F14091C10182E1489FFF
:10187000800111240C5A1E4FA8014D5F5F4FD80103
:101880008C9112966C910E948906F8018181815099
:101890008183882309F04AC08091C1018F5F8093C2
:1018A000C1018091C101863008F440C01092C1018D
:1018B0003DC080914001882361F480913F018F5F9A
:1018C00080933F01803228F010923F0181E08093A5
:1018D000400180913F01882351F060E00E94E30CB9
:1018E000892B29F480913F0180933E011CC0809197
:1018F0003E010E94370DFC01009751F080818093DA
:101900003E018185863031F4CF010E94670702C015
:1019100010923E01809140018F5F80934001809141
:101920003E01882319F080640E94760284E180934E
:101930002A0326960FB6F894DEBF0FBECDBFCF9117
:10194000DF911F910F91FF90EF90DF900895EAECE7
:10195000F1E0482F50E020E030E08081882311F44E
:1019600021E030E02417350711F480E008953C961B
:1019700082E0EA38F80779F781E0089580918A02D9
:1019800090918B0208959C01EAECF1E00CC08285F5
:10199000882309F48185883029F481819281821716
:1019A000930739F03C9682E0EA38F80781F7E0E0E7
:1019B000F0E0CF01089580ECEAECF1E0DF011D9248
:1019C0008A95E9F70895CF93DF93382F81508F31AF
:1019D000D0F5CAECD1E004C088818317B1F12C9610
:1019E00082E0CA38D807C1F7662369F120E0CAEC63
:1019F000D1E025C08881882301F5388382E089877A
:101A000000D000D000D0EDB7FEB7319681E790E06E
:101A1000ADB7BEB712969C938E9311973283138203
:101A2000248315820E9489118DB79EB706960FB642
:101A3000F8949EBF0FBE8DBF08C02C962F5F92E01A
:101A4000CA38D907B8F2C0E0D0E0CE01DF91CF911B
:101A50000895882319F420E030E003C00E94E30CCD
:101A60009C0130938B0220938A02C90108950F9341
:101A70001F93182F882311F401E005C0803210F065
:101A80000FE101C0082F1F5F103208F011E0812F15
:101A900060E00E94E30C9C01101711F0009799F38D
:101AA000C9011F910F91089580E090E008958FEF94
:101AB0009FEF0895089580E0089580E090E00895F4
:101AC0008FEF9FEF0895682F87FF9CC080911603CA
:101AD00090E001969C0143E0220F331F4A95E1F705
:101AE000280F391F24533D4F80911A0390911B03F7
:101AF00082179307E1F4809116038F5F809316039A
:101B000080911603883010F01092160390911603FE
:101B100080911703981759F4809117038F5F809372
:101B2000170380911703883010F01092170310925A
:101B30001B0310921A03109219031092180380913C
:101B40001001681721F481E0809320038DC010926A
:101B50002003262F30E02F773070482F50E02417D5
:101B6000350729F06F3F19F08F3F09F07DC0809154
:101B7000160379E0879FC001112484539D4F9093F1
:101B80001B0380931A032417350709F06DC0909149
:101B90001403809115039817D1F480911403879F43
:101BA000D0011124AA56BD4FEDE8F2E081918D934A
:101BB00082E0E639F807D1F7809114038F5F8093B4
:101BC000140380911403863010F010921403809156
:101BD000150329E0829FC00111248A569D4F9093DE
:101BE000190380931803809115038F5F8093150369
:101BF00080911503863010F01092150389E08093D0
:101C00008C0232C020912003213029F0213060F174
:101C1000263050F515C082E080932003603419F41B
:101C20001092210321C0613419F4209321031CC0B8
:101C3000623419F0633491F483E08093210314C07B
:101C4000E22FF0E08091210390E002968E179F072B
:101C500044F0E65EFC4F8081681719F01092200373
:101C600003C02F5F2093200380912003882329F055
:101C700060932B0310922C0321C0E0911803F09184
:101C800019033097A9F0819180932B0310922C03B4
:101C9000F0931903E093180380918C028150809394
:101CA0008C02882359F4109219031092180306C06D
:101CB0008FEF9FEF90932C0380932B03E0911A03F7
:101CC000F0911B03309749F083E0E431F80728F4E2
:101CD0006193F0931B03E0931A030895109220037D
:101CE0001092190310921803089590911403809193
:101CF000150320E0981709F421E0822F08958FB78B
:101D0000F8949091140320911503492F50E0421B41
:101D100051098FBF57FF02C04A5F5F4F25E030E097
:101D2000241B350BC9010895DC014FB7F8942091AD
:101D300014038091150330E090E0019728173907CC
:101D400041F080911403853039F480911503882384
:101D500019F44FBF80E008959091140389E0989F93
:101D6000F0011124EA56FD4F90E08D9181939F5F21
:101D70009930D9F7809114038F5F80931403809179
:101D80001403863010F0109214034FBF81E00895C1
:101D9000DC01EDE8F2E08D91819382E0E639F8070D
:101DA000D1F708959C01009739F14FB7F8949091BD
:101DB000160380911703981721F44FBF20E030E0FD
:101DC0001BC09091170389E0989FF0011124E45300
:101DD000FD4FD90190E081918D939F5F9930D9F7A4
:101DE000809117038F5F80931703809117038830CA
:101DF00010F0109217034FBFC90108958FEF9FEFA6
:101E000090932C0380932B030E945E01262F2F7743
:101E100020931F03F7E09695879577956795FA9538
:101E2000D1F7262F2F7720931E03E7E0969587950D
:101E300077956795EA95D1F7262F2F7720931D0385
:101E400057E096958795779567955A95D1F76F776F
:101E500060931C030E941E0308958091240388232D
:101E600019F01092240381E008952091220330910B
:101E700023039093230380932203C9010895809143
:101E800010010895FF920F931F93DF93CF93CDB767
:101E9000DEB729970FB6F894DEBF0FBECDBFDA01CB
:101EA000A89580911001806889836A83FE0133962A
:101EB0009E01275F3F4F109721F08D918F77808390
:101EC00001C010823196E217F307A9F78E010F5F68
:101ED0001F4FC8010E94CE108987F02E012F8F2D31
:101EE000902F0E94940E8823D1F381E029960FB69B
:101EF000F894DEBF0FBECDBFCF91DF911F910F9140
:101F0000FF9008952F923F924F925F926F927F922F
:101F10008F929F92AF92BF92CF92DF92EF92FF92F9
:101F20000F931F93DF93CF93CDB7DEB729970FB6EB
:101F3000F894DEBF0FBECDBF809110018F3F09F036
:101F40006FC00E945E019B01AC0139014A0177E03C
:101F500095948794779467947A95D1F78FE790E07A
:101F6000A0E0B0E0682279228A229B2259016A010E
:101F70006EE0D594C794B794A7946A95D1F7A82238
:101F8000B922CA22DB2279018A0195E115950795CC
:101F9000F794E7949A95D1F787E090E0A0E0B0E05D
:101FA000E822F9220A231B238FE7282E312C412C0B
:101FB000512C222233224422552234C0A8958A81F2
:101FC000843081F5CE0101960E94E510882351F1FD
:101FD0008E8190E0A0E0B0E0281639064A065B0644
:101FE00009F58D8190E0A0E0B0E0681679068A06D8
:101FF0009B06C1F48C8190E0A0E0B0E0A816B90681
:10200000CA06DB0679F48B8190E0A0E0B0E0E81628
:10201000F9060A071B0731F489818F778093100135
:1020200081E007C0CE0101960E94D20E892B31F6C5
:1020300080E029960FB6F894DEBF0FBECDBFCF91DA
:10204000DF911F910F91FF90EF90DF90CF90BF90A5
:10205000AF909F908F907F906F905F904F903F9048
:102060002F900895FF920F931F93DF93CF93CDB7D7
:10207000DEB729970FB6F894DEBF0FBECDBF8091B3
:1020800010018F3F69F50E94820F882399F180919A
:1020900010010E94A9032EC0C8010E94E5108823E8
:1020A00021F1298130E02F7730708091100190E08C
:1020B0002817390711F40E946F038A81863019F4BA
:1020C000F092240312C0E0912203F0912303309791
:1020D00019F0C801099509C0C8010E94C20305C0D2
:1020E0008E010F5F1F4FFF24F394C8010E94D20E90
:1020F000892B91F629960FB6F894DEBF0FBECDBF9F
:10210000CF91DF911F910F91FF9008950F931F932F
:10211000DF93CF93CDB7DEB729970FB6F894DEBF24
:102120000FBECDBF209110012068298323E02A83B0
:10213000282F2F772B83880F892F881F990B919534
:102140008F778C83862F8F778D83852F86958695C5
:102150008E8367FF02C080648E83CA01E3E0969598
:102160008795EA95E1F78F778F83842F8295807723
:1021700088878E010F5F1F4FC8010E94CE1089878C
:10218000C8010E94C80E29960FB6F894DEBF0FBE94
:10219000CDBFCF91DF911F910F910895FC0120E0F9
:1021A00090E037E08191982780E097FF03C0990F76
:1021B000932701C0990F8F5F8830B9F72F5F2830C0
:1021C00089F797FD9095892F08950F931F938C01A0
:1021D0000E94CE1020E0F8019085891709F421E0D3
:1021E000822F1F910F910895FC01862F8F77828394
:1021F000852F8695869566956074862B8383CA01A4
:1022000023E0969587952A95E1F78F778483429509
:10221000407745830895FC01862F8F778083660F72
:10222000672F661F770B71956F77618308950F9302
:102230001F93CF93DF93082F162FEA0102C00E944D
:102240006E00802F612FAE010E94420F8823B9F3E8
:10225000DF91CF911F910F910895DF93CF9300D01D
:1022600000D000D0CDB7DEB7FE01319696E0DF0199
:102270001D929A95E9F74983AF010E94171126969E
:102280000FB6F894DEBF0FBECDBFCF91DF9108959A
:102290009B01AC018091260390912703A091280314
:1022A000B091290382179307A407B50798F080918E
:1022B000260390912703A0912803B091290360E0A1
:1022C000821B930BA40BB50B80509041A040B040F3
:1022D000A0F412C08091260390912703A0912803B7
:1022E000B091290360E0281B390B4A0B5B0B20508F
:1022F000304F4F4F5F4F08F061E0862F0895E82F71
:10230000F0E0EF70F070E857FF4FE4918E2F90E00F
:102310000895A0E0B0E0EFE8F1E10C943C14FE0178
:10232000359661917191A0913003B091310313966C
:102330008C911397886013968C93809130039091C1
:102340003103AF010E94AF11E0913003F0913103EE
:102350002381277F23832096E2E00C945814ABE07E
:10236000B0E0E5EBF1E10C942C143C012B015A0197
:10237000FC0117821682838181FD03C06FEF7FEF1E
:10238000C6C19AE0892E1E010894211C311CF3015C
:102390002381F20123FD859123FF81912F01882361
:1023A00009F4B2C1853239F423FD859123FF81916F
:1023B0002F01853229F490E0B3010E94A213E7CFE8
:1023C000982FFF24EE249924FFE1FF15D0F09B32D3
:1023D00069F09C3228F4903259F0933291F40EC097
:1023E0009D3249F0903369F441E024C052E0F52A6F
:1023F00084E0F82A28C098E0F92A25C0E0E1FE2A06
:1024000022C0F7FC29C0892F80538A3070F4F6FE71
:1024100005C0989C902C1124980E15C0E89CE02CC7
:102420001124E80EF0E2FF2A0EC09E3229F4F6FCD9
:102430006BC140E4F42A07C09C3619F450E8F52A31
:1024400002C0983649F4F20123FD959123FF919142
:102450002F01992309F0B8CF892F8554833018F0C4
:102460008052833038F444E050E0A40EB51E5FE3A0
:1024700059830FC0933631F0933779F0933509F0D3
:1024800056C020C0F5018081898342E050E0A40E4F
:10249000B51E610101E010E012C0F501C080D180DD
:1024A000F6FC03C06FEF7FEF02C0692D70E042E0E1
:1024B00050E0A40EB51EC6010E9497138C015FE781
:1024C000F52214C0F501C080D180F6FC03C06FEF87
:1024D0007FEF02C0692D70E042E050E0A40EB51E0F
:1024E000C6010E948C138C0150E8F52AF3FE07C048
:1024F0001AC080E290E0B3010E94A213EA948E2DEC
:1025000090E008171907A8F30EC0F601F7FC8591B3
:10251000F7FE81916F0190E0B3010E94A213E110D8
:10252000EA94015010400115110579F7EAC094367C
:1025300011F0993669F5F7FE08C0F5012081318167
:102540004281538184E090E00AC0F501808191814D
:102550009C01442737FD4095542F82E090E0A80E5F
:10256000B91E9FE6F92257FF09C050954095309556
:1025700021953F4F4F4F5F4FE0E8FE2ACA01B90156
:10258000A1012AE030E00E94CE13D82ED21840C01C
:10259000953729F41F2D1F7E2AE030E01DC01F2D26
:1025A000197F9F3661F0903720F4983509F0ACC060
:1025B0000FC0903739F0983709F0A6C004C028E062
:1025C00030E00AC0106114FD146020E130E004C066
:1025D00014FD166020E132E017FF08C0F5016081AC
:1025E00071818281938144E050E008C0F5018081CF
:1025F0009181BC0180E090E042E050E0A40EB51E65
:10260000A1010E94CE13D82ED2188FE7F82EF12206
:10261000F6FE0BC05EEFF522D91438F4F4FE07C0C5
:10262000F2FC05C08FEEF82202C01D2D01C0192D4D
:10263000F4FE0DC0FE01ED0DF11D8081803319F413
:1026400099EEF92208C01F5FF2FE05C003C08F2D6E
:10265000867809F01F5F0F2DF3FC14C0F0FE0FC049
:102660001E1510F09D2C0BC09D2C9E0C911A1E2D3A
:1026700006C080E290E0B3010E94A2131F5F1E1506
:10268000C0F304C01E1510F4E11A01C0EE2404FFCB
:102690000FC080E390E0B3010E94A21302FF1DC0AF
:1026A00001FD03C088E790E00EC088E590E00BC014
:1026B000802F867891F001FF02C08BE201C080E29A
:1026C000F7FC8DE290E0B3010E94A21306C080E304
:1026D00090E0B3010E94A2139A94D914C0F3DA9443
:1026E000F101ED0DF11D808190E0B3010E94A21374
:1026F000DD20A9F706C080E290E0B3010E94A2139A
:10270000EA94EE20C1F743CEF30166817781CB01D5
:102710002B96E2E10C944814FC0105906150704046
:102720000110D8F7809590958E0F9F1F0895FC019A
:102730006150704001900110D8F7809590958E0FF0
:102740009F1F08950F931F93CF93DF938C01EB018D
:102750008B8181FF1BC082FF0DC02E813F818C8148
:102760009D812817390764F4E881F9810193F98381
:10277000E88306C0E885F985802F0995892B31F417
:102780008E819F8101969F838E8302C00FEF1FEF82
:10279000C801DF91CF911F910F910895FA01AA27E7
:1027A000283051F1203181F1E8946F936E7F6E5F94
:1027B0007F4F8F4F9F4FAF4FB1E03ED0B4E03CD042
:1027C000670F781F891F9A1FA11D680F791F8A1F25
:1027D000911DA11D6A0F711D811D911DA11D20D08C
:1027E00009F468943F912AE0269F11243019305D46
:1027F0003193DEF6CF010895462F4770405D419337
:10280000B3E00FD0C9F7F6CF462F4F70405D4A3383
:1028100018F0495D31FD4052419302D0A9F7EACF4B
:10282000B4E0A6959795879577956795BA95C9F77A
:1028300000976105710508959B01AC010A2E06946D
:102840005795479537952795BA95C9F7620F731F26
:10285000841F951FA01D08952F923F924F925F9263
:102860006F927F928F929F92AF92BF92CF92DF92A0
:10287000EF92FF920F931F93CF93DF93CDB7DEB705
:10288000CA1BDB0B0FB6F894DEBF0FBECDBF099499
:102890002A88398848885F846E847D848C849B84F0
:1028A000AA84B984C884DF80EE80FD800C811B81FE
:1028B000AA81B981CE0FD11D0FB6F894DEBF0FBE2D
:0A28C000CDBFED010895F894FFCF9D
:1028CA0000808000800000808000008000808000FE
:0228DA00FF00FD
:00000001FF
